:040000008A11A52A92
:1004480064008001840A0406031900340406252A7E
:10045800F90079088312031386008A115A228A1137
:100468000D30F800F80B362A08007E088A007F084D
:10047800820039228A118000840A04087D06031943
:100488000034FF0A0319FE0A3D2A013083120313C0
:1004980086008A118C228A110A3083120313D50030
:1004A8000030D6008A1173228A11080083120313C0
:1004B80085141030F700F70B5F2A640083120313CA
:1004C80005151030F700F70B672A64008312031331
:1004D80005111030F700F70B6F2A64000800832A13
:1004E800F930F7006400F70B762A7A2A6400FF30A7
:1004F80083120313D5070318D60AFF30D6078312D1
:10050800031356085504031D8A2A8B2A742A0800E7
:100518008312031385101030F700F70B912A64003B
:100528008312031305151030F700F70B992A64009E
:100538008312031305111030F700F70BA12A64008A
:1005480008007030840077308A1124228A118313BE
:100558002030840051308A1124228A11C030FD00D5
:100568000230FE00C030FF00A03084008A113D2216
:100578008A1183018A11F32E303431343234333402
:1005880034343534363437343834393441344234F9
:100598004334443445344634EE34ED34EB34E734F4
:1005A800DE34DD34DB34D734BE34BD34BB34B73449
:1005B8007E347D347B347734F22A5508840056081B
:1005C8008A1100238A118A112C228A110130831280
:1005D8000313D5070318D60A0030D607831203136E
:1005E8005508840056088A1100238A110038031D13
:1005F800FE2AFF2AE12A0800FE00FE1F082B8313AB
:100608007E188317000808000408FE0003308A00DB
:100618007E0882070034013400340A34003464341C
:100628000034E834033410342734533455344D340B
:100638003D3400344D34413458343D34003425348D
:10064800643400340030F7000030F80083120313DC
:10065800511C2F2B302B362B5308F7070318F80A99
:100668005408F80701300310D30DD40DFF3E031DC5
:10067800372B01300310D20CD10CFF3E031D3E2B4B
:1006880052085104031D492B4A2B2A2B7808D20102
:10069800D2077708D101D1070800031000300318EA
:1006A8000130F6007608B03E840083130008740613
:1006B800031D5F2B602B672B7608A03E8400000883
:1006C80083120313B2007608013EF600103076025A
:1006D800031C6F2B702B562B8312031332088600D2
:1006E8006430D5000030D6008A1173228A110800C0
:1006F800F030831603138600831203130608F500EF
:100708007508F039AF0074080F39F40074082F0425
:10071800F4000608F5007508F039AF002F08F03A24
:100728000319972B982B992B8D2B03100030031846
:1007380001308316031386008A1151238A1183120C
:1007480003133208B100B0010314B00D080083127E
:1007580003135B085A040319B22BB32BE32BF901DB
:100768000314F90DC22B01300310DA0DDB0DFF3E27
:10077800031DB82B0130F8007808F907DB1FC52BDB
:10078800C62BB72B5B085902031DCC2B5A085802FD
:10079800031CCF2BD02BD62B5A08D8025B08031C7E
:1007A800D903D90201300310DB0CDA0CFF3E031D1C
:1007B800D72B0130F902031DE22BE32BC62B590876
:1007C800D901D9075808D801D80708000030831282
:1007D8000313D1000030D200570856040319F52B33
:1007E800F62B2E2CD3010314D30D052C0130031046
:1007F800D60DD70DFF3E031DFB2B0130F700770800
:10080800D307D71F082C092CFA2B01300310D10D60
:10081800D20DFF3E031D0A2C57085502031D162C46
:1008280056085402031C192C1A2C212C5608D402E1
:100838005708031CD503D502511401300310D70CF7
:10084800D60CFF3E031D222C0130D302031D2D2C94
:100858002E2C092C5208D501D5075108D401D407EC
:10086800080038308312031386008A118C228A11FB
:10087800053083120313D5000030D6008A11732285
:100888008A1138308312031386008A118C228A1148
:100898002130F800F80B4E2C3830831203138600F1
:1008A8008A118C228A112130F800F80B592C383023
:1008B8008312031386008A118C228A112130F800D2
:1008C800F80B642C01308312031386008A118C22E2
:1008D8008A11323083120313D5000030D6008A11F2
:1008E80073228A110D308312031386008A118C2219
:1008F8008A112130F800F80B7F2C0630831203137D
:1009080086008A118C228A112130F800F80B8A2C73
:100918000800031000300318013083120313B000DD
:100928001830831603138500F03086008113EF30EA
:10093800F40074088312031386000430AD00E22C1F
:100948007408F800F9017808D5007908D600023053
:10095800D7000030D8008A11E9248A118313831242
:1009680003135508F400740886000530D5000030DC
:10097800D6008A1173228A1183120313061EC52C0E
:10098800C62CD22C861EC92CCA2CD22C061FCD2CC4
:10099800CE2CD22C861BD12CD22CD52C8A117C2380
:1009A8008A11831203133008013A031DDC2CDD2C55
:1009B800DF2C3108E82C2D08FF3EAD00AD08031DE3
:1009C800E62CE72CA42C8D2C08000310003003180B
:1009D800013083120313D200D81FF32CF42CFC2C03
:1009E800D709D809D70A0319D80AD2010314D20D96
:1009F800D61FFF2C002D092DD509D609D50A0319B4
:100A0800D60A0130F7007708D2060030D30000304C
:100A1800D400580857040319122D132D4B2DD1015A
:100A28000314D10D222D01300310D70DD80DFF3E30
:100A3800031D182D0130F7007708D107D81F252D81
:100A4800262D172D01300310D30DD40DFF3E031DA5
:100A5800272D58085602031D332D57085502031C2D
:100A6800362D372D3E2D5708D5025808031CD603BE
:100A7800D602531401300310D80CD70CFF3E031DC7
:100A88003F2D0130D102031D4A2D4B2D262D520832
:100A9800031D4F2D542DD309D409D30A0319D40AA1
:100AA8005408D601D6075308D501D5070800831284
:100AB8000313D5000030D3000030D400550884005B
:100AC80083130008D100840A0008D200413056067A
:100AD8005704031D702D712DB52D0030F000003026
:100AE800F1007108803AF70080307702031D7E2DEF
:100AF80005307002031C812D822D832DAC2D7008CA
:100B0800F70077078312031355078400831300083F
:100B1800F800013084070008F90053087807D3006B
:100B280054080318540A7907D4000130F007031851
:100B3800F10A0030F1077108803AF7008030770237
:100B4800031DA82D05307002031CAB2DAC2D832D81
:100B5800831203135408D701D7075308D601D607C1
:100B68000B2E0130F0000030F1007108803AF700D8
:100B780080307702031DC22D05307002031CC52D7D
:100B8800C62DC72D032E7008F700770783120313AD
:100B98005507840083130008F80001308407000813
:100BA800F9005208803AFA007908803A7A02031D5F
:100BB800DF2D780851020318E22DE32DF02D70087F
:100BC800F70077078312031355078400831300087F
:100BD800D100840A0008D2000130F0070318F10A96
:100BE8000030F1077108803AF70080307702031D62
:100BF800FF2D05307002031C022E032EC72D831211
:100C080003135208D701D7075108D601D6070800A1
:100C180083120313E500C130E000D72E6608253A99
:100C28000319172E182E242E6608DC006508840088
:100C38005C08831380000130DC005C08E507D72ED0
:100C48000310003003180130DF000001013883165B
:100C58000313C0070001FF3840078A1109238A11CE
:100C680083120313E600003A0319EA2E643A0319C3
:100C7800412E0D3A0319412ED72E600884008313A4
:100C88000008E200840A0008E3000230DC005C0887
:100C9800E007E31F502E512E5A2E0330DC005C086B
:100CA800DF04E209E309E20A0319E30AE60103148F
:100CB800E60D6608DC005C07013EDE008A110923A8
:100CC8008A11DD00DE0A5E088A1109238A11DE0016
:100CD8005E086302031D722E5D0862020318752EFA
:100CE800762E772E812E0130DC005C08E607660838
:100CF800053A031D802E812E5D2E5F0803390319E6
:100D0800862E872E922E2D30DC00650884005C0824
:100D1800831380000130DC005C08E5076608E10009
:100D2800CD2E6308D501D5076208D401D407610820
:100D3800DC005C07013EDD008A1109238A11D60018
:100D4800DD0A5D088A1109238A11D7008A11EA236E
:100D58008A118313831203135508D901D90754083C
:100D6800D801D8070A30DA000030DB008A11AB233B
:100D78008A118313831203135808303EE60066086D
:100D8800DC00650884005C0880000130DC005C0839
:100D9800E507FF30DC005C08E1076108FF3A031D46
:100DA800D62ED72E952E0001013883160313C007BF
:100DB8000001FF3840078A1109238A11831203139F
:100DC800E600E608031DE92EEA2E122E0310650838
:100DD8008400003003180130831380000800981342
:100DE8000730831603139C000310003003180130EA
:100DF8009D0003100030031801309B001830850057
:100E080083120313051003100030031801308316F2
:100E180003138600031000300318013083120313F4
:100E280086008A1135248A118A1149228A113E3096
:100E38008A112C228A110030F0000030F10071086C
:100E4800803A83120313E70080306702031D2E2FB8
:100E580005307002031C312F322F332F962F8A1141
:100E680049228A113E308A112C228A118A118D2436
:100E78008A1183120313E700E8016708F200680883
:100E8800F30072088A112C228A118A118D248A1182
:100E980083120313E700E8016708AB006808AC0099
:100EA8002B088A112C228A11E83083120313D500EB
:100EB8000330D6008A1173228A117208D03E831239
:100EC8000313D10073080318013EFF3ED2000A3015
:100ED800D3000030D4008A1126238A118312031309
:100EE8002B0883135107E7002C0803182C0A520714
:100EF800E8006708D03EA90068080318013EFF3ED5
:100F0800AA007008E7006707343E840029088000BB
:100F1800840A2A0880000130F0070318F10A00301B
:100F2800F107232F8A1149228A112A308A112C228B
:100F38008A118A118D248A1183120313E700E801AC
:100F48006708F2006808F30072088A112C228A11D7
:100F5800730883120313D701D7077208D601D6077F
:100F680034308A115B258A118313831203135708BF
:100F7800AC01AC075608AB01AB078A1149228A11AC
:100F8800413072067304031DCA2FCB2FD52F0B30A7
:100F980083120313D5000030D6008A11E0228A118B
:100FA800DE2F103083120313D5000030D6008A11CB
:100FB800E0228A11153083160313C000831203132D
:100FC8002C0883160313C201C207831203132B08CC
:100FD80083160313C101C1074C308A110C268A11EC
:100FE8004C3083120313D5008030D6008A11E022DA
:080FF8008A11FD2F8A11002867
:00000001FF
